S1048000007B
S123C000C787C769C790C7C4C76FC777C77FC7D2C7EAC7E2C7F2C844C83AC82EC833C84D42
S123C020C865C8B3C875C885C895C93BC95BC967C97BC78DCA5EC991C9A6C99BCABACAC614
S123C040CAD1C9C3C9AFC9CDC9D7C9E7CA28CA54CA63CA7FCA8ECA9DCA34CA44CA19C9FF5B
S123C060CAE6CAEACAF0CB01CB14CB07CB4ACB1CCB5ACBBDCBD2CBE0CBF2CB95CB9FCB7866
S123C080CBA8D77AD726D750D768D78DD7A0D7B2D7BDD7D5D7FAD80AD7ABD825D839D84472
S123C0A0D81AD84FD85AD865D877D885D893D735D8BBD8E0D8CBD8A1DCF2DDD0DDD4DE1947
S111C0C0DA8ECBABCBB4DA67DA9DDAAE0000D1
S123C500FCFF0227358E00FFBDE0CF1AB3FF022608CC0000FDFF022021BDDB82CEC52DBD27
S123C520DCE1B67F0084C088C027F720134D454D4F5259204641554C54008EFEFF7F003C6D
S123C5408D392016B67F0084038103260D8E00FF0FBDE0CFFDFF027EE06BB67F00848088D8
S123C5608027037EC712B680004A26F7CC8001CEC300ED008600A7097EC712CE002A4FA7D3
S123C58000088C003926F8CE1000860AB77F00970E86FF9722972397249725CC07C0DD265E
S123C5A01C39801D282086B0A72B860CA72D86079739BDDB82CC0000DD0CDD12DD14860835
S123C5C0970BCCC110DD16DD18DD1A8620B7C6F8CEC300C6208640A7098FC300108F5A26C0
S123C5E0F6CEC300DF08CCC200ED00CCFE00ED04C30001ED02830100ED06860AA708862084
S123C600A709EF0CEF0EDC0CC30001DD0CED0ABDDAAECEC639A6002706BDDB540820F6CE25
S123C62010001C200118CE3000180926FC1D20011D0008CC0000DD2639496E74657261631F
S123C6407469766520432020205620322E383220362F31312F39370A008D6B8D748161258B
S123C660F881732604863E2068368D513C18388D4C328172270D8177270F81632711816255
S123C680271B39A6008D4A2010188FE700200A188FA400A700EA00E700863E2034188F37FD
S123C6A03C32331B331B97015D270C8D19A7009B019701085A26F496018D1620DC8D073647
S123C6C08D0416328F39B6102E842027F9B6102F39F6102EC48027F9B7102F39DE08A60874
S123C6E0970A1AEE00EE0218E600F7C6F11808FCC000FDC6F6BDFFFF20ED8620B7C6F8DC9D
S123C700088FED021AEF00A60981402604EE0CDF0839963C260CCE10001F2E2005BDC659A2
S123C72020F0120B02ECDE08EE0EDF088CC3002607DC1EC30001DD1EA609810026D4BDC62F
S123C740DC810027CD814027C9812027048602200286048D0220BB9701940B910126013940
S123C76096019A0B970B7EC6D1EC02A300201CEC02A400E4012014EC02AA00EA01200CECAF
S123C78002A800E8012004EC00E302ED020808398D26A601E6033DDD00A600E6033DDB00D1
S123C7A0D700EC013DDB00D7007D000727064F5F930020D7DC0020D37F00078D6308088DF7
S123C7C05F090939BDC7B8EC023CEE0002DF003820D7EC00A3022705CC000020AECC000123
S123C7E020A9EC02A3002EF520EEEC02A3002DED20E63CEC002B1C260438080839373686EC
S123C80005B7C807EC02380027030926FA380808ED00394F5FA30037368604B7C80720E4D0
S123C8206D002A094F5FA300ED007300073963006301394F5FA300ED0039EC002705CC0008
S123C84001ED0039EC0027F64F5FED0039EC02E306DD00E601E905A600A904ED04DC00ED3A
S123C86006C6043A39EC06A302DD00E605E201A604A20020E6EC06A302E605E201A604A22C
S123C880002D1E2025EC02A306E601E205A600A2042D0E2015EC06A302260FEC04A300265E
S123C8A009C6063ACC0001ED0039C6063ACC0000ED00397F0007BDC9513CC6043ABDC95106
S123C8C0CE0000DF0038A603E6073DDD02A603E6063DD301DD01960089009700A602E607EE
S123C8E03DD301DD01960089009700A603E6053DD300DD00A602E6063DD300DD00A601E600
S123C900073DD300DD00EC033DDB00D700A602E6053DDB00D700A601E6063DDB00D700A697
S123C92000E6073DDB00D700C6043ADC02ED02DC00ED007D000727028D0139CC0000A30298
S123C940DD00C600E2018600A200ED00DC00ED02396D002A058DE47300073918EC00180850
S123C96018080909ED003918EC020909ED0018EC00180818081808180820E718E600183A7B
S123C98018A60009A70018095A26F518E600183A393CCDEE00E600384F20C38FCDEE00EE87
S123C9A0028F0909ED008FCDEE00EE008F20AF18E6003C3AEC00DD00EC02380909ED00DC0F
S123C9C000209D18E6003C3AEC003820933CA601CDEE00A70020083CEC00CDEE00ED0018F6
S123C9E0083818080808393CEC00DD00EC02CDEE00ED02DC00ED0038C6043A57183A39EC1A
S123CA0000DD00EC02D70718E6003C3AD607ED02DC00ED0038080820C9EC00D70118E6006D
S123CA203C3AD601ED0020B9A6013CEE02273FA70038202AA601B7CA403CEE0227301C0076
S123CA40FF38201AA601B7CA503CEE0227201D00FF38200AEC003CEE022713ED0038080871
S123CA60080839EC00DD00EC023CEE0426063886057EDE25ED02DC00ED0038080820DFEC29
S123CA80003CEE0227E8E70038ED02080839EC003CEE0227D9ED0038ED02080839EC00DDC2
S123CAA000EC023CEE0427C6ED02DC00ED0038EC02ED04DC00ED020808393CEE0027AFE6A0
S123CAC0004F38ED00393CEE0027A3EC0038ED00393CEE002798EC00DD00EC02380909ED90
S123CAE002DC00ED003918EE00391AEE00080839EC00260618EE00080839180818080808E7
S123CB0039EC0026EF20F3EC0027EFCC0001ED0018EE0039EC0026E218EE0039EC00DD00CD
S123CB2018EC00DF04D3048F1AEE002705DC00ED0039DE088640A7098621B7C6F8EC0C1AE4
S123CB40EE0E8FCDEF0C1AEF0E3918EC00DF00D3008F1AEE0027DB080839EC00DD00EC02DF
S123CB60DD0218EC00DF04D3048F1AEE0227C3DC00ED00DC02ED0239DF00DE08DC00A30678
S123CB80CDA300250718081808DE00391809DE0086047EDE258F18E3008F18081808393CC6
S123CBA0323318E3007EC95EEE0039EC00DD3A0808180839DC3A0909ED00180839EC003C43
S123CBC0EE021AA300382427E302C30002ED02080839EC003CEE021AA3003824120520E8EF
S123CBE0EC003CEE021AA300382404050520D97EDE1FEC003CEE021AA3003824F218A6009D
S123CC0018083D20C33CBDD696CE00003CDF41DF437F00451830CDEE06A600BDCD5D252878
S123CC20812D260B73004508A600BDCD5D2519812E260B08A600BDCD5D24037ECCCB313173
S123CC40BDD6A038860F0D39A600BDCD5D2477BDCCDC0824F37C0041A60008BDCD5D25F572
S123CC60812E260AA600BDCD5D24030820F681452707816527037ECD1F08A600BDCD5D25D7
S123CC8015812D2706812B270520B318630008A600BDCD5D24A8803018A70108A600BDCD71
S123CCA05D241418E601585818EB015880301B18A701088126228718A601186D002A01403E
S123CCC09B4197412059812E26A408A600BDCD5D249C8D0808258D7A004120EF9642974786
S123CCE0DC43DD4805790042252C057900422526D3483696429947974232251A05790042BD
S123CD00DD432512E600C0304FD343DD43964289002503974239DC48DD439647974239CDC2
S123CD20EF06CE0041BDCD88272C964118A70186969741BDCD69186D01271B2A0BCECD93DD
S123CD40BDD6C91860012006CECD97BDD6C9BDCDA7186A0126F83131BDD6A0383981302598
S123CD6006813922020D390C39CE00418D1A27147D00422B0FDC437A0041270A057900428B
S123CD802AF5DD430C390D393736EC002602EC023233393DCCCCCD41200000BDD043BDD652
S123CDA096BDCF12BDD6A07D004127057D0046260ACC00009745DD41DD43399645984A97B8
S123CDC04596419B462A0924168606CEFFFF2009250D8607CE0000DF44DF41DF430D398BA1
S123CDE0829741CE00003C3C30BDCE206D002B0B69036902690169007A00416D032A13A659
S123CE00024CA702260CC601E3002404467C0041ED0038DF42329744317D004127B45F395B
S123CE209649D6443DA7019648D6443DE300ED009649D6433DE300A70324026C026F006FD7
S123CE40019647D6443DE302ED029648D6433DE302ED0224026C019649D6423DE302ED0222
S123CE6024026C019647D6433DE301ED0124026C009648D6423DE301ED0124026C00964710
S123CE80D6423DE300ED0039BDD696CED3C2BDD6C97D0045270373004ABDCF44BDD6A04F4D
S123CEA0D641C17F24035F201B53C3FF902F178FDC422001040926FC7D00452A074353C322
S123CEC000012A020C3986090D39CC0000DD004FD641C17F24035F203353C3FFA02F2F8F3D
S123CEE096445FDD00DC422007047600007600010926F67D00452A14730000730001435340
S123CF00DE0008DF002605C300012A020C3986090D39BDD32ACE0049964680972A1BC60341
S123CF208B082A096F00095A26F66F0039C6804A2B035720FAE400E7008D028D07964A880C
S123CF40FF974A399641260EDC46DD41DC48DD43964A97455F397D004627F9D645D84A9021
S123CF60462510811822ED183C36CE004718CE0042201740811822D0183C369646974196ED
S123CF804A9745CE004218CE004717363636A8003617A8013617A8023630A606E706168443
S123CFA0074CC4185454543AE6034A27095666026601660020F45618A602A900974418A6AE
S123CFC001A901974318A600A902974230A6062B15245A7600427600437600447C004126DE
S123CFE04CCCCDC92053251B73004570004424087C004326037C004270004324037C0042F6
S123D0007000427D00422B2526139641800823269741DC4327207F0044DD4220E67A004189
S123D02027147800447900437900422AF01AEE07C6093A355F39CCCDD21AEE07ED07C60744
S123D0403A3539964A984597457D0046260586087ECDCB7D004126055F7F0045399641904D
S123D0604624052B057ECDD22B1F8B7E9741DC4293472B182606964490492B10DC420476D8
S123D0800044DD427C004126037ECDC9DC42DE470826010903183C18DE42DF423CCE0000FA
S123D0A03C3C309649D6433DA703BDCE4A18DF42DC43A301DE4703DF437F00423838323334
S123D0C01838D342DD425F393CCE0041BDCD88260738CC3000ED0039DE413CDE433C9645B9
S123D0E036BDD696CE00003C3C3C1830CDEE0F86207D004527057F0045862DA70008CDEFC3
S123D10000CED232BDD6C9BDD2362E19CED22EBDD6C9BDD2362E16186A02CECD97BDD6C98C
S123D120BDCDA720DC186C02CECD9320F0CED3C2BDD6C9BDCF44D641C07F50CB17200A7445
S123D14000427600437600445A26F4860118A70318A6028B082B0A810824064A18A703868C
S123D16002800218A702186D032E15862ECDEE00A70008186D0327058630A70008CDEF00A8
S123D180CED219860718A705186F04DC43A301DD439642A20097422505186C0420EDDC43E2
S123D1A0E301DD439642A900974218A6048B303CCDEE00A70008186A032605862EA70008D7
S123D1C0CDEF0038080808186A0526BCCDEE0009A600813027F90818E602272A8645A700D0
S123D1E008862BA7005D2A0550862DA70008CDEF004FCE000A02378FCB30CDEE00E700083D
S123D20033CB30E700086F00383838BDD6A032974538DF4338DF4138390F42400186A000BA
S123D22027100003E800006400000A000001497423FE4B18967F964A2A12D6452A0EDC4672
S123D2401A93412617DC481A934320109145260CDC411A93462605DC431A93480784F42461
S123D260028A080639CE008EC3000026057ECDD209052AFCDD427F00448F9745D7415F393F
S123D2804D2AE24353C30001CEFF8E20DBCE009EC30000261118DE0026037ECDD20978005E
S123D2A00179000059492AF5DD42960097448F9745D7415F394D2AD57300007300014353BB
S123D2C0DE0008DF002603C30001CEFF9E20C1CE0041BDCD882601397D00452A04860A0D3E
S123D2E039BDD696860436DE433CDE413C18308D399646807E4C2A03442003448B7E97465E
S123D300BDD043BDCF447A00418D1F18EC00DD4118EC02DD43186A0426E6DC46DD41DC48C4
S123D320DD43383831BDD6A05F39DC41DD46DC43DD489645974A39BDD696CED491BDD6C92C
S123D340BDD043BDD6A0DC411A8385B32B0B7D004526037ECDC97ECDD2BDD6969645367FC9
S123D3600045BDCF12DC4627068086544C26FC5C37CED3A6BDD656CED3A2BDD6C92003BD6D
S123D380CDA7306A0026F832324D2A0CBDD32ACED5EABDD6B0BDD043BDD6A05F39BDD69628
S123D3A020EA402DF8543638EF1D37D00D0139500D013AB60B613C0888893D2AAAAB3E2AAB
S123D3C0AAAB3F0000003F8000003F800000FFBDD3EBBDCDA77ED3468D11BDD696CED491FB
S123D3E0BDD6C9BDCDA7BDD6A05F3996452704860C0D39964127F8BDD6963C3C30BDD6E1B8
S123D4004FD641C07F2A0143BDD280CED48DBDD6C9BDCDA730BDD6C9BDD6E1867F97463C0C
S123D4203C30BDD6EFCED5EABDD6B0BDCF4430BDD6C9BDD6E1CED489BDD6B0BDCF4430BD2F
S123D440D6C9BDD04330BDD6E1BDD32ABDCDA7CED46CBDD65630BDD6C9BDCDA7383830BDB9
S123D460D6C9BDCF443838BDD6A05F393E1D89D93E3A2E8C3E638E393E9249253ECCCCCDC6
S123D4803F2AAAAB40000000FFBF8000003F3172183EDE5BD9860E0D39860D0D39BDD69626
S123D4A09645367F0045CED5EABDD6C9BDD2362F07BDD39D86FF20014F363C3C30BDD6E13B
S123D4C0BDD32ABDCDA7CED4F4BDD65630BDD6C9BDCDA73838324D270CCED4F0BDD6C9739E
S123D4E00045BDCF44BDD640329745BDD6A05F393FC90FDBBCE2DD1B3D70F0F1BD888889FB
S123D5003D9D89D9BDBA2E8C3DE38E39BE1249253E4CCCCDBEAAAAAB3F800000FFBDD696AE
S123D5204F2005BDD69686F036CED608BDD6C92003BDCF44964526F92003BDCF39BDD236FC
S123D5402EF88D61240930A6002B04880FA7008D54240930A6002A04880FA7008D472407F4
S123D56030A60088F0A700CED64EBDD6C9BDCDA7BDD32ABDCDA73C3C30BDD6EFA6042A0545
S123D580CED5EF2003CED5DABDD65630A6044724037300454D2B06BDD6C9BDCDA7383831C0
S123D5A0BDD6A05F397A0046BDD2362E020C397C0046730045BDCF447A00460D39BDCF12B4
S123D5C0DC41DE46DD46DF41DC43DE48DD48DF439645D64A974AD7455F393638EF1DB95024
S123D5E00D013C088889BE2AAAAB3F800000FF37D00D01BAB60B613D2AAAABBF0000003F1E
S123D600800000FF40490FDB43B40000BDD696BDD32ABDD523BDD5C0BDD51DBDD043240789
S123D620BDD6A0860B0D39BDD6A05F397FFFFFFFBDD696CED64EBDD6C9BDCDA7BDD6A03981
S123D640BDD696CED65220EECED6047ED6B03C8EFA3142652EE18FDE413CDE433C8F964591
S123D660363CCC0000DD41DD43DD44201030A602974AEC03DD48EC05DD46BDCDA730EE00A9
S123D680BDD6C9BDCF4438C6043A3CA6004326DD30C6073A3539383C3C8F3037367ED6EF32
S123D6A0300808BDD6C938313131316E00CED5EA7F0045EC02DD43EC00052403730045979A
S123D6C04127020D56D7425F397F004AEC02DD48EC0005240373004A974627020D56D74790
S123D6E039DC43ED02DC4158D1454656ED0039DC48ED02DC4658D14A4656ED00397F004564
S123D7005F397D00422705CC7F80DD414F5FDD43397D004227037300455F39BDD6C90808ED
S123D7200808BDD6B0393C183CEC00BDD280183838090920AC3C183C0808BDD6B00909EE85
S123D74000BDD0C8183838EC00ED0408080808393C183CBDD6B0BDCECA18383824037EDE7F
S123D76025ED00DC00ED02393C183CEC02DD00EC00BDD2B51838387ED6E13C183CBDD6B074
S123D780BDCE9F18383824037EDE25205D3C183CBDD71BBDCF44183838080808087ED6E1C2
S123D7A03C183CBDD71BBDCF3920EBA6008880A700393C183CBDD71BBDCDA720093C183C9F
S123D7C0BDD71BBDD04318383824037EDE25080808087ED6E13C183CBDD71BBDD2361838ED
S123D7E038260CCC0001080808080808ED00390808080808086F006F01393C183CBDD71B11
S123D800BDD2361838382BDB20E53C183CBDD71BBDD2361838382ECB20D53C183CBDD71BF3
S123D820BDD3CF20A13C183CBDD6B0BDD2CF18383824037EDE257ED6E13C183CBDD6B0BD9E
S123D840D34620EA3C183CBDD6B0BDD33720DF3C183CBDD6B0BDD3EB20D43C183CBDD6B0F3
S123D860BDD3D820C93C183CBDD6B0BDD49D0736BDD630320620B73C183CBDD6B0BDD6409D
S123D880BDD51D20A93C183CBDD6B0BDD640BDD523209B3C183CBDD6B0BDD640BDD60C2091
S123D8A08D8602E6019D4B080839BDDB9AA600BDDC7EA601BDDC7E08082003BDDB9AA6007F
S123D8C0BDDC7EA601BDDC7E080839BDDB9A3CEE008602E60027059D4B0820F738080839A8
S123D8E0183CDF00BDDAFA1A830051240C8621B7C6F8DE001838180939DE00DC00C300021F
S123D900E300DD02830002DD04DE02EE000808A60026037EDA55812527037EDA4308A60068
S123D9208166261BDF02DE0409093CBDD6B0380909DF04CEC100BDD0C8CEC1007EDA3581B9
S123D94064267DDF0218CEC100DE040909DF04EC022A0C862D18A7001808CC0000A302CE68
S123D960000A02378FCE000A02378FCE000A02378FCE000A02378FCE000A0237183C3886CE
S123D98001335D27064FCB30E70008334D27045D27064FCB30E70008334D27045D27064F9A
S123D9A0CB30E70008334D27045D27064FCB30E7000833CB30E700085FE700CEC100207584
S123D9C08178262ADF02DE040909DF04A602BDDC64BDDB42257217BDDB42256CA603BDDC68
S123D9E064BDDB42256217BDDB42255C206181632611DF02DE040909DF04A603BDDB4225F0
S123DA0047204C8162261EDF02DE040909DF04E60318CE00085886308900BDDB42252918C2
S123DA200926F2202A8173261ADF02DE040909DF04EE020808A6002708BDDB42250A082085
S123DA40F4200CBDDB422409860ABDDB542006DE02087ED90FDE00DC00C30002E3008FCCEE
S123DA600000ED001838393CDC14C300011A931426FBC30001CE0000081A931426FA8F3818
S123DA800909ED00CC000C0909ED007EC790090909090FDC14ED02DC120EED0039EC0008AF
S123DAA0083C183CEE00AD00183838ED00390F3C183CB6103C84402605CEFF002003CEBF74
S123DAC0003CC6C03A18CEE0E11AEF0008083C32324D26F538CCC500EDFECCDE9FEDE2CCE6
S123DAE0DE92EDE0CE10006F226F248600A7211C23181C22181838380E39960B84082707BE
S123DB00CC00F0DD062016DC1893162307830001DD062009CC00F09316D318DD06960B847D
S123DB20102705CC00F02012DC1A931623058300012007CC00F09316D31A1A93062302DC3F
S123DB4006393736BDDAFA1A83000224040D323339322001370F3CDE16088CC2002603CEFC
S123DB60C110DF16A700960B840827119C18260DDE18088CC2002603CEC110DF1838330C66
S123DB800E398D79CC00389D4BC60C9D4B8D198601970F8608971C4F971DCC00019D4BC6FC
S123DBA0069D4BC68F9D4B39CC00409D4B8602CEDBBDE6009D4B088CDBFD26F639000A1F63
S123DBC01F0E04000000001111110F010E00000000000C040800000F11110F010E00000C4C
S123DBE00C000C0C0000000C0C000C0408020006020202120C00000A0E04000000CEDC12C9
S123DC0018CE004BA60018A7000818088CDC6426F339FF009ACE10000F1D3C201D0010B741
S123DC20009C6F078104260F8601B710041C0010A6031D001020228601B710041C0010A65A
S123DC40031D0010848026EF86FFA707B6009CA704E7031C00101D00101C3C20FE009A0EE6
S123DC603900000036840F8B30813A2B028B071632444444448B30813A2B028B0739BDDC0A
S123DC8064371686029D4B339D4B39CE000A02378FCE000A02378FCE000A02378FCE000A53
S123DCA002378FCE000A02379D4BCC00019D4BCC00079D4BCC008F9D4B860233CB309D4B4E
S123DCC033CB309D4BC62E9D4B33CB309D4B33CB309D4B33CB309D4BC66D9D4BC6739D4BD0
S123DCE039CC00029D4B8602E60027059D4B0820F739183CDF00CC7FFFDD04CEC3001AEE60
S123DD000E188CC3002607CCE400DD06200518EC04DD06EC0693063CDE00A300382B091AEC
S123DD2093042E04DF02DD04188CC3002705183C3820CBDC041A837FFF260486012015CE9B
S123DD40C310A609814027158FC300108F8C620026F08602DE00183818097EDE253C183867
S123DD60DE02EE0E1AEF0CCDEF0EDE021AEF0ECDEF0CEC0683000118ED04C30001DE00A361
S123DD800018ED06A60318A708EC0418ED00860018A709DC0CC30001DD0C18ED0ADC00E35E
S123DDA006C30008EE068F09DF0018DF0218EE0436A60018A7003209180983000126F1DEB0
S123DDC00218081AEF02DE0009DC0CED00183839862020513CEC00DD00CEC300EC0A1A937D
S123DDE000270EEE0E8CC30026F238CC0001ED00399C082604387ECB32183C8640A709868B
S123DE0021B7C6F8EC0C1AEE0E8FCDEF0C1AEF0E183838CC0000ED00398621B7C6F8391805
S123DE2009860320003CDE084D2602861FA70997018621B7C6F8960181202431CEDE6FA63E
S123DE40002708BDDB4225F70820F44FD601C00A25034C20F9CB0A8B30BDDB4225FB178BD4
S123DE6030BDDB4225FB860ABDDB4225FB38390A52554E54494D45204552522000CE100044
S123DE80DC28E316ED161D237FB610008880B710003BCE1000DC26E31EED1E1D23F73BCEC3
S123DEA01000CC07D0E31CED1C1D23EFA622368408A7220EDE1408DF142605DE1208DF1212
S123DEC07A000A26058621B7C6F886049D4B848027037EDFAC9615843F2640960F810122AD
S123DEE03A0F4FC6CF9D4BDC1E1A8300642D0BCC0000DD1E961C880C971C961C84082704AD
S123DF00C6002002C60786029D4B4FD611C1102502CB30CA809D4B0E7EDFAC9639840126EC
S123DF20037EDFAC960F8102245EDE1A9C16277C088CC2002603CEC110DF1AE600960F81B7
S123DF40002634C10A26068601970F205F9611811F27594C9711811126074F37C6C09D4B52
S123DF6033C120250CC17F2208CEDFEEC0203AE60086029D4B20358101260DD710FCDFDC3B
S123DF809D4B8602970F2024810A2712CEDFDCD60F3AEC009D4B960F8B02970F200E860057
S123DFA0970F86019711D610C10A26B5D60E963984042720C6FF96229B3D973D5696239BA7
S123DFC03E973E5696249B3F973F5696259B40974056D40EF77F0032B710223B000100069C
S123DFE000CF020000020011495557777FFF202122232425262728292A2B022D2E2F3031A0
S123E000323334353637383904053C3D3E3F404142434445464748494A4B4C4D4E4F505138
S123E02052535455565758595A5B5C5D5E5F60616263646566036869066B6C6D6E6FF0F174
S123E04072737475767778017A7B7C7D7E7F18CE03E8180926FCCE10001F000433CC1BE688
S123E0601F00042C83000126F7203937368D56CC00029D4BCEE0998602E60027059D4B087C
S123E08020F732BDDC7E32BDDC7E8602C6299D4BCE10001C28204F06CF2A48616C74656492
S123E0A02A2028008D1FCEE0B5BDDCE1CE10001D23FB8D163B2D504F57455220474C495460
S123E0C043482D20008601979839860E979839CE80004F5FE3008FC300028F8CFF0226F410
S105E0E0393BC6
S123BFC0E0E1E0E1E0E1E0E1E0E1E0E1E0E1E0E1E0E1E0E1E0E1E0E1E0E1E0E1E0E1E0E14D
S123BFE0DE92DE9FE0E1E0E1E0E1E0E1E0E1E04EE0E1E0E1E0E1E0E1E0E1E0E1E0E1C50051
S123FFC0E0E1E0E1E0E1E0E1E0E1E0E1E0E1E0E1E0E1E0E1E0E1E0E1E0E1E0E1E0E1E0E10D
S123FFE0DE92DE9FE0E1E0E1E0E1E0E1E0E1E04EE0E1E0E1E0E1E0E1E0E1E0E1E0E1C50011
S105FF020000F9
S105FF000251A8
S9030000FC
